:020000040000FA
:10000000E7280530AA00A530AB00AB0B0528AA0BEA
:10001000032800348600003066000515851005149D
:100020000510FF3066000511851405140608AF00A1
:10003000AF1705100514861F1F2805101A28051074
:100040003228860000306600051185100514051061
:10005000FF30660085140514861F302805102B28F4
:10006000051000342F1C0034AF1C00342F1D003449
:10007000AF1D00343930AF07AF172F082128831385
:1000800010088D0203184B2801308E0203184B28EC
:100090008F02031C831711088E02031853280130A6
:1000A0008F02031C831712088F02031C831700346E
:1000B00010088D07031C5F288E0F5F288F0A110818
:1000C0008E0703188F0A12088F0700340730AA0022
:1000D000193084002F308000840AAA0B6B280F305F
:1000E000920042309100403090003F20990A3A300F
:1000F000190603196E2A831F7528582001309200B3
:1001000086309100A03090003F209A0A831F8428F7
:100110005820920127309100103090003F209B0A18
:10012000831F8E28582003309100E83090003F2034
:100130009C0A831F972858209101643090003F202B
:100140009D0A831F9F2858200A3090003F209E0A56
:10015000831FA62858200D089F079F0A00343730B8
:10016000620010306500851105118F018101960133
:10017000051505110C08AA008515FA30AB00C62834
:1001800000000000000000000000000001089602CE
:10019000031DCC280000CE2803188F0A960000000B
:1001A00000000000AB0BC028AA0BBD288511010878
:1001B0008E009602031CDE28031D8F0A8D018D031D
:1001C0000515051101080E060319DF280034850105
:1001D00010306500860100306600012001200120FA
:1001E0003830860005140120051005140120051083
:1001F000051401200510061221200C3021200130A9
:1002000021200630212020300A2020300A204A30C8
:100210000A2061300A206E300A206B300A206F30CD
:100220000A2020300A2053300A2061300A2075301D
:100230000A2070300A2065300A2072300A206C30A3
:100240000A200630AC00C830AD000120AD0B2529D6
:10025000AC0B2329013021200630212020300A2038
:1002600020300A2020300A2020300A2053300A2073
:1002700035300A2035300A2057300A2054300A2001
:1002800020300A2020300A2020300A2020300A2086
:1002900020300A2020300A200630AC00C830AD00E3
:1002A0000120AD0B5029AC0B4E2901302120063026
:1002B000212020300A2020300A2020300A2020303F
:1002C0000A205A300A2061300A2063300A206E303A
:1002D0000A2069300A206D300A206F300A20203051
:1002E0000A2020300A2020300A2020300A20203026
:1002F0000A200630AC00C830AD000120AD0B7D29CE
:10030000AC0B7B29013021200630212014308C00D9
:10031000AF20662030301906031D922930301A06AE
:100320000319D129823021200230AA00193084001B
:1003300030300006031DA22920300A20840AAA0BAF
:100340009829A72900080A20840AAA0BA2292E307E
:100350000A200530AA0000080A20840AAA0BAB294B
:1003600020300A2047300A2048300A207A300A20FC
:1003700020300A2020300A20862914308C00AF203B
:10038000662030301906031D922932301A020318F4
:10039000922930301A06031DD12930301B0603196B
:1003A000FA29823021200530AA001930840030302B
:1003B0000006031DE12920300A20840AAA0BD72950
:1003C000E62900080A20840AAA0BE1292E300A2017
:1003D00000080A20840A00080A2020300A204D3034
:1003E0000A2048300A207A300A2020300A202030A3
:1003F0000A20BD29C8308C00AF2066203030190695
:10040000031DBD2932301A020318BD2930301A06E7
:10041000031D0E2A30301B0603194A2A8230212080
:100420000430AA001930840030300006031D1E2A53
:1004300020300A20840AAA0B142A232A00080A2042
:10044000840AAA0B1E2A2E300A2000080A20840AD9
:1004500000080A20840A00080A2020300A204D30B3
:100460000A2048300A207A300A2020300A20203022
:100470000A20FA29C8308C00AF20662030301906D7
:10048000031D0E2A30301A06031D0E2A32301B02BD
:1004900003180E2A823021200730AA001930840068
:1004A00030300006031D5A2A20300A20840AAA0B85
:1004B000502A5F2A00080A20840AAA0B5A2A2030F0
:1004C0000A204B300A2048300A207A300A20203097
:1004D0000A2020300A2020300A203A2A0130212028
:1004E000843021204F300A2076300A2065300A20DF
:1004F00072300A2066300A206C300A206F300A20E1
:0A05000077300A20023021208629FE
:00000001FF
